:10000000000002308A002E2AA101A117B400FE30A0
:10001000E7203408E728C600B71F10282D30E72056
:10002000B90F1728B80F1728B70A0319B70ABE0166
:10003000BF01C001C101B7176A30B6070310B70C82
:10004000B80CB90CC10CC00CBF0CBE0CB60F1E28EE
:1000500039083602B907B60238083702B807B702BE
:10006000A4016A202E30E720C70103103E0DB9001D
:100070003F0DB800400DB700410DB600C70D03108D
:10008000B90DB80DB70DB60DC70D3E08B9073F083D
:1000900003183F0FB80740080318400FB70741087F
:1000A0000318410FB6070318C70F0310B90DB80D99
:1000B000B70DB60DC70D4708303EE7203908BE0022
:1000C0003808BF003708C0003608C100C60B342806
:1000D00003106729A0112408031D7128A0150A30F8
:1000E000A4003908A8003808A7003708A600360879
:1000F000A500A301B001AF01AE010A30AD0012218D
:10010000A30A23082402031D7A282D08031DA01129
:10011000A01D8C28240B8F282D08303EE720A40B2F
:1001200071286729A3002408031967292308E720F9
:10013000A4039328B20086110611831686110611B6
:100140000F30860583123208A018C4283E30A6005E
:100150008030FE203330B100D8201330A600883024
:10016000FE20D8206430FD20D8206430FD202230CD
:10017000B100D8202030C3200C30C3200630C3206B
:10018000A0143208C4282014B100201CD228061163
:10019000033C031CD728D7200730A600D030FE2010
:1001A000031408002014FE3C0319E5280615201C42
:1001B000201086150F3086053108F0398604861127
:1001C000B10E2018D8283230FD2032086729A11B33
:1001D0009A280800B100B10DB10D310D3839C13880
:1001E0009F003230FD201F151F19F4281E08B7008C
:1001F00083161E088312B6006729A601E83EA500F3
:10020000A609FC30031C0729A50703180429A50724
:100210000000A60F042925180D29A51C112900008E
:1002200011290800BA01BB01BC01BD012130AB009E
:100230003929BA0DBB0DBC0DBD0D2D083A022E0893
:10024000031C2E0F3B022F08031C2F0F3C0230080B
:10025000031C300F3D02031C3929BD002D08BA02D2
:100260002E08031C2E0FBB022F08031C2F0FBC02ED
:100270000314A50DA60DA70DA80DAB0B19293D085C
:10028000B0003C08AF003B08AE003A08AD0067295B
:10029000A601AA01A900AE01AD011030B100260DE2
:1002A000AD0DAE0D2908AD022A08031C2A0FAE02BF
:1002B000031861292908AD072A0803182A0FAE0779
:1002C0000310A50DA60DB10B4F29250808008313B7
:1002D0008312031308003F08BC004306CA00C2088B
:1002E0000319D329BE080319D6294208BE027F305C
:1002F00003187E29BE07031CD5298129BE070318D0
:10030000D8294108BA004008BB00BC17C3171830F1
:10031000C900C101C001BF018F2903189B294508ED
:100320003A024408031C440F3B024308031C430FDA
:100330003C02031CA6294508BA024408031C440FCA
:10034000BB024308031C430FBC020314C10DC00DC4
:10035000BF0DBA0DBB0DBC0DC90B8D29BF1BB82934
:10036000BE080319D529CA0CBE03C90ACA0D8D29B6
:100370000318C6294508BA024408031C440FBB02EF
:100380004308031C430FBC02031CD229C10FD2290E
:10039000C00FD229BF0FD229BF0CC00CC10CBE0A9E
:1003A0000319D829DF29C815D9294815BE01DB2929
:1003B000C814FF30BE00C101C0018030BF00CA1B9D
:1003C000E229BF136729C001C101CA13F629CA1364
:1003D000C11FF629C109C009BF09BE09BE0FF52911
:1003E000BF0FF529C00A0319C10ACA179630C90000
:1003F000C1080319042A0830C9073F08BE00400895
:10040000BF004108C000192AC008031D192A08307E
:10041000C9023F08031D152A0830C9023E08031D02
:10042000142A4108C900232ABE01C0003E08BF00AB
:10043000BE01C01B212A0310BE0DBF0DC00DC90394
:10044000192ACA1FC0133E08C1004908BE0040084F
:10045000C9003F08C0004908BF0067298301403038
:10046000C800A00183168117FF309C009F01073050
:100470008500C0309F00831200308A01EA20CB0043
:100480003708CC008030A1008C308A0104209A30DB
:10049000C5009930C4004C30C3008630C2004C08FF
:1004A000BF004B08BE008A01E3218A016B2141088D
:1004B000B9004008B8003F08B7003E08B600023057
:1004C0008A010B20FE308A019A2040308A019A204E
:1004D0008030A1000830A40000308A019220003052
:1004E0008A019A200630A40010308A019220003040
:1004F0008A019A2000308A019A200630A400143024
:100500008A01922000308A019A2000308A019A20C4
:100510000630A40015308A0192208A11CD2A243099
:100520004D028A110318982A4D08CF008A119A2A81
:100530002430CF004F08A50003308A014821CE00A7
:10054000A6014F08A500AA010330A9008A014B218A
:100550002D08D000013050028A110318B32A500828
:10056000D1008A11B52A0130D1008030A1008A0162
:1005700004204E08A40003308A0192205108A400F0
:1005800050088A01922051084E07B60036080C3CEC
:10059000A40020308A01922008004C08A6004B08D5
:1005A000A500AA011F30A9008A014B21CD008A01B4
:0A05B0008F228A013B2A8A01DB2A10
:02400E00323F3F
:00000001FF
